:050B1E00C10401080004
:10010000C2AFE4F5A8F5E8C28C438901758CFD7592
:100110008A65D28CF5B8F5F8C2BBD2B8D2A9C28D27
:10012000C28FD2ADD288C289D2AFF517C2C5C2C0C4
:10013000C2C3C2C1C2C2C2C41207C2750C0A7529A9
:1001400005D2A83002FDC202D20975110175120153
:10015000D513057513FAB2C00528E52870020527E6
:10016000C39410E52794274008E4F527F5281203E7
:1001700057300D051204A3920D200E031203F33025
:100180000E30E50ED394144029E50C6025150CE5DE
:100190000C701F750C01E50D6013D50D10C20E78A3
:1001A00072E6600E16E6600A1203CA8005C21112DA
:1001B0000495E517C39401400AE517D3940B500347
:1001C000D38001C392C4E517C3940C400AE517D34A
:1001D00094165003D38001C392C2E5106009151034
:1001E000E5106003D38001C392C3E50F6009150FCA
:1001F000E50F6003D38001C392C1200A03020143CB
:10020000C20A43871075FF32120BEFEF54C0700320
:0A0210000201431207C2020143225B
:10021A00AE07EE600FE4FF74562FF8E6B50601222A
:07022A000FBF08F37FFF2264
:0C023100E4FF7F087856E4F608DFFC22AA
:10023D00AE07E4FDED25E025E0242EF8E6B5060C2D
:10024D00ED25E025E0242EF9E4AF01220DBD0AE4F1
:03025D007F0022FD
:100260008F2B8B2CAC05AF0412023DEF602604F8F7
:10027000E6FE30E312EF2402F8E6652C6016EF0488
:10028000F8EE54F7F6800DEF2402F8E6B52C05AF32
:1002900004120324E4FEEE25E025E0242EF8E665B2
:1002A0002B7033EE25E025E02430F8E6652C600E57
:1002B000EE25E025E0242FF8E64408F6800CEE2534
:1002C000E025E0242FF8E64410F6EE25E025E024B2
:1002D0002EF9E4AF01220EBE0ABCE4FEEE25E025B5
:1002E000E0242EF8E660090EBE0AF1E52B5407FE65
:1002F000EE25E025E0242EF8A62BEE25E025E024CF
:100300002FF8E4F6EE25E025E02430F8A62CEE25C3
:10031000E025E02431F87684EE25E025E0242EF96E
:04032000E4AF012223
:10032400E4FEEE25E025E0242EF8E6B50720E4F609
:10033400EE25E025E0242FF8E4F6EE25E025E02480
:1003440030F8E4F6EE25E025E02431F8E4F60EBEBC
:030354000AD022AA
:10035700E4FFEF25E025E02431F8E6602C16E6708F
:1003670028EF25E025E0242EF8E4F6EF25E025E048
:10037700242FF8E4F6EF25E025E02430F8E4F6EF43
:0E03870025E025E02431F8E4F60FBF0AC52278
:10039500E509D39414502CE50A75F00BA42400FF4D
:1003A5007D7D7B0A120FB1E50A75F00BA4240AF8CE
:1003B5007414F2050AE50AC394144003E4F50A052A
:0503C50009D322C32250
:1003CA00E509D394145020E50A75F00BA42400FF24
:1003DA007D687B0B120FB1050AE50AC3941440032A
:0903EA00E4F50A0509D322C3223F
:1003F300E50960257F68E50B75F00BA42400FD7B00
:100403000B120FA6050BE50BC394144003E4F50B85
:0B0413001509D20E750D02D322C32282
:10041E00787DE624DE24FD500E24F524FD500824BC
:10042E00F124FD50028049850A2B85092CE52C60AC
:10043E003FE52B70047F148004E52B14FF8F2BEF08
:10044E0075F00BA42402F8E2787F66701FEF75F04A
:10045E000BA42400F8E2787D667011EF75F00BA402
:10046E002400FF7D7D7B0A120FB1D322152C80BD97
:04047E0012039522AE
:10048200200908A20092111207E422A2009211127E
:03049200049522AC
:0E049500120C015007301102D205D322C322EF
:1004A300785EE624C07003020557147003020584C6
:1004B3001470030205AA2422B42F0040030207C0CC
:1004C3009004CAF82828730205570205840205AA76
:1004D3000205F60206420206820206930206C402DF
:1004E30006D50206ED020716020743020743020779
:1004F300C00207530207C00207C00207C00207C0B9
:100503000207C00207750207C00207C00207C00244
:1005130007C00207C00207C00207C00207C00207E4
:10052300C00207C00207C00207C00207C00207C01B
:100533000205F60206420206820206930206C4027E
:1005430006D50206ED020716020743020743020718
:10055300C00207537860E6FF7862E6FD08E6FB1207
:1005630002608F2AA807E804F8E64404F654FEF66E
:100573007F877D5E7B0A120FBCC2111207E402075C
:10058300C07860E6FF12023D8F2AEF70030207C0B6
:1005930004F8E64404F67F877D5E7B0A120FBCC233
:1005A300111207E40207C07860E6FF12023D8F2AAA
:1005B300EF70030207C004F8E630E0030207C0A8A7
:1005C30007E82403F876847F877D5E7B0A120FBCDD
:1005D300C2111207E4E52A04F8E620E3030207C088
:1005E300C2AD7F7D7D5E7B0A120FBC12041ED2ADAD
:1005F3000207C07860E6FF12023D8F2AEF70030204
:1006030007C004F8E630E0030207C0A807E82403A4
:10061300F876847F877D5E7B0A120FBCC2111207B6
:10062300E4E52A04F8E620E3030207C0C2AD7F7DB8
:100633007D5E7B0A120FBC12041ED2AD0207C07886
:1006430060E6FF12023D8F2AEF70030207C0240306
:10065300F876847F877D5E7B0A120FBCC211120776
:10066300E4E52A04F8E620E3030207C0C2AD7F7D78
:100673007D5E7B0A120FBC12041ED2AD0207C07F3F
:10068300877D5E7B0A120FBCC2111207E40207C00A
:100693007860E6FF12023D8F2AEF70030207C00461
:1006A300F8E630E0030207C0A807E82403F87684DD
:1006B3007F877D5E7B0A120FBCC2111207E402071B
:1006C300C07F877D5E7B0A120FBCC2111207E40252
:1006D30007C0E52A2403F876847F877D5E7B0A12B0
:1006E3000FBCC2111207E40207C07860E6FF1202D2
:1006F3003D8F2AEF70030207C004F8E630E00302DF
:1007030007C07F877D5E7B0A120FBCC2111207E40C
:100713000207C07860E6FF7862E6FD08E6FB120296
:10072300608F2AA807E804F8E64404F654FEF67F2F
:10073300877D5E7B0A120FBCC2111207E40207C059
:100743007F877D5E7B0A120FBCC2111207E4806DA6
:100753007860E6FF12023D8F2AEF606104F8E6201D
:10076300E05B7F877D5E7B0A120FBCC2111207E438
:10077300804B7860E6FF12023D8F2AEF603F7F8750
:100783007D5E7B0A120FBCC2111207E4E52A240323
:10079300F876847862E6FFE52A2402F8A607E52ABC
:1007A30004F8E654FEF6C2AD787D7634087602A8E6
:0F07B3002AE6787FF6E408F612041ED2ADC322C0
:1007C2007F01120BF57F437D1C7B1A120B247FFFE6
:1007D2007DFF120B5B7FC0120BEC7F2A120BF5D24E
:0207E2000822EB
:1007E400301102D203752BFAC2AD120BEFEF30E2D7
:1007F400117F87120BA07FC1120BECD2AD75100FC5
:0E080400D322D2ADD52BE17FC2120BECC32262
:10081200301002D2037525FAC2AD120BEFEF30E2AF
:10082200117F73120BA07FC1120BECD2AD75100FAA
:0E083200D322D2ADD525E17FC2120BECC3223A
:03000B00020840A8
:10084000C0E0C0D0C28C758CFD758A65D28CA201C7
:10085000B392015002D20230B20BE50EC394FF50A6
:0F08600007050E8003E4F50ED20AD0D0D0E032A7
:03002B0002086F59
:10086F00C0E0C0F0C083C082C0D0C000C001C002D1
:10087F00C003C004C005C006C007120BF2EF20E092
:10088F0003020B037F7D120BD07F04120BEC750F4D
:10089F000F787DE624E0B42B004003020B03900891
:1008AF00B4F8282873020935020B030209850209DF
:1008BF00980209AB020B03020B03020B03020B039B
:1008CF00020B03020935020B03020B03020B030297
:1008DF000B03020B030209BE0209E0020A1B020B03
:1008EF0003020A40020AAC020B03020AD5020ADA1B
:1008FF00020B03020B03020B03020B03020B030297
:10090F000B03020B03020935020B030209850209CF
:10091F00980209AB020B03020B03020B03020B033A
:10092F00020B03020935787FE6FF12023D8F23EF9A
:10093F00601E04F8E6FF20E017787376340876021D
:10094F00A823E67875F6EF548008F6C21012081245
:10095F00787FE6FF12021AEFF47003020B0378732D
:10096F007634087602787FE67875F6087602C2103C
:10097F00120812020B03787FE6FF12023DEF70039D
:10098F00020B0312041E020B03787FE6FF12023DD7
:10099F00EF7003020B0312041E020B03787FE6FFB6
:1009AF0012023DEF7003020B0312041E020B0378B9
:1009BF007FE6FF12023D8F23EF7003020B0304F853
:1009CF00E6FF20E203020B03547FF612041E020B14
:1009DF0003787FE6FF12023D8F23EF7003020B03B4
:1009EF0004F8E6FF20E203020B0330E006787D7681
:1009FF0036800BEF5418FEBE0804787D7636E5235B
:100A0F0004F8EF546BF612041E020B03787FE6FF17
:100A1F0012023D8F23EF7003020B0304F8E6FF2051
:100A2F00E203020B034480F654EAF612041E020B93
:100A3F0003787FE6FF12023D8F23EF601504F8E67F
:100A4F00FF20E20620E00312041EE52304F8E6442B
:100A5F0001F6787FE6FF12021AEFF47003020B0320
:100A6F00E4F52474562524F8E6FF12023D8F23EF98
:100A7F00601D04F8E6FF20E0164401F6787D763419
:100A8F00087602A823E6787FF608760212041E0580
:100A9F0024E524C3940840CB1202318057787FE6B7
:100AAF0024FC6013240424FA500824FD24FC500273
:100ABF00804212041E803D7880E6FF12023DEF60F7
:100ACF003312041E802E12041E8029787FE6FF1237
:100ADF00023D8F23EF601D12041EE4F524747F2561
:100AEF0024F8E6FF74562524F8A6070524E524B458
:100AFF0008EB8000D007D006D005D004D003D00279
:0F0B0F00D001D000D0D0D082D083D0F0D0E0324F
:100B24008F2A8D2B8B2C120BFB8F2DEF20E006448C
:100B340001FF120BF57F06AD2A120BE27F07AD2BE6
:100B4400120BE27F08AD2C120BE27F017D80120BA9
:070B5400E2AF2D120BF522A8
:100B5B008F2A8D2B120BFB8F2CEF20E0064401FF0D
:100B6B00120BF57F04AD2A120BE27F05AD2B120B96
:070B7B00E2AF2C120BF52282
:100B8200ED601AEF4420F5DB0BEBAE0270010A14A4
:0E0B9200F5828E83E0F5DAAF051DEF70EB22E1
:100BA000A2AF920BC2AF8FD875DB8A0000A20B9266
:020BB000AF2272
:100BB200ED601AEF4420F5DB0BEBAE0270010A1474
:0E0BC200F5828E83E5DAF0AF051DEF70EB22B1
:100BD000A2AF920CC2AF8FD875DB940000A20C922A
:020BE000AF2242
:050BE2008FDB8DDA221B
:050BE7008FDBAFDA22F4
:030BEC008FD9227C
:030BEF00AFD8225A
:030BF200AFD92256
:060BF500E4F5DB8FDA22BB
:060BFB00E4F5DBAFDA2295
:100C0100D20EE517700A30A807E50EC394145002FE
:100C1100C322C28E53890F438910758DFF758B9B3B
:0A0C2100D28EC2A8C28FD2ABD3223C
:03000300020C2BC1
:100C2B00C0E0C0D020B22FE511602B300928C28E56
:100C3B0053890F438910758DFF758B0AD28EC28F26
:100C4B00D2ABC2A8D20FE517700375170CE517C30B
:0B0C5B00940C4002C2B4D0D0D0E032B4
:03001B00020C666E
:100C6600C0E0C083C082C0D0C000C28EE517B417F2
:100C7600004003020F76900C83F8282873020CC8F4
:100C8600020CE4020CF8020D12020D35020D4502AB
:100C96000D55020D79020DAF020DC4020DD8020DDD
:100CA600EC020E0F020E25020E3B020E4B020E5FE9
:100CB600020E84020E9D020EE0020F1E020F480273
:100CC6000F5720B209C2ABC289D2A8020F81758D17
:100CD600F2758BFAD28ED2C5751701020F7F758D0C
:100CE600E0758BC1D28EC2C5751702C289D2A80221
:100CF6000F7F758DFD758B65D28E30B203020E00A7
:100D0600200F03020E00751703020F7F30B2030295
:100D16000E00758DE5758BF6D28E7869E6540F2434
:100D260002F516751468751501751704020F7FC252
:100D3600C5758DFD758BCFD28E751705020F7FD2C7
:100D4600C5758DFE758B63D28E751706020F7FA84B
:100D560014E6551524FFB392C5500A758DFE758BA2
:100D660063D28E8008758DFD758BCFD28E75170771
:100D7600020F7FA2C5B392C5500A758DFE758B63AF
:100D8600D28E8008758DFD758BCFD28EE515251513
:100D9600F515700FD51606751709020F7F7517081A
:100DA600020F7F751706020F7FC2C5758DF5758B0D
:100DB60095D28E0514751501751704020F7F758D72
:100DC600E0758BC1D28E75170AC2C5C289D2A80238
:100DD6000F7F758DF8758B2FD28E20B21D300F1AAE
:100DE60075170B020F7F20B211750C32E4F517C28E
:100DF6000EC2ABC289D2A8020F7FE4F517750C1993
:100E0600C2ABC289D2A8020F7F758DFC758B17D233
:100E16008EC2B430B203020F6675170D020F7F3013
:100E2600B203020F66758DE5758BF6D28E75170EB9
:100E3600D2B4020F7FD2C5758DFA758BCAD28E7564
:100E4600170F020F7FC2C5758DE0758BC1D28E75E7
:100E56001710C289D2A8020F7F758DFE758B15D229
:100E66008ED2B430B203020F66200F03020F6675EE
:100E7600145E75160C751501751711020F7F758DA9
:100E8600FE758B15D28EC2B430B206751712020FDC
:100E96007F751713020F7F758DFE758B15D28ED257
:100EA600B430B203020F66A814E64515F6E515251B
:100EB60015F515701FD51610C28E758DE5758BF656
:100EC600D28E751715020F7F751714C28EC289D27E
:100ED600A8020F7F751711020F7F758DFE758B1592
:100EE600D28ED2B430B279A814E515F456F6E515CB
:100EF6002515F515701DD5160FC28E758DE5758BEA
:100F0600F6D28E7517158071751714C28EC289D2E6
:100F1600A880667517118061758DFE758B15D28E4A
:100F2600D2B420B23B0514E514D394675032E516CB
:100F3600B40A07785FE6540FF51675150175171193
:100F46008037D2C5758DF5758B95D28E751716803F
:100F560028D20DE4F517C2C5C2ABC289D2A8801942
:100F6600E4F517750C32C2ABC289D2A8D2B4800997
:100F7600C2ABC289D2A8E4F517C20FD000D0D0D038
:060F860082D083D0E032AE
:100F8C008E838F828D01E709F0A3DBFA228C838D8F
:100F9C00828F01E0F709A3DBFA228F008D01E3F6C3
:100FAC000809DBFA228F008D01E7F20809DBFA222F
:0B0FBC008F008D01E7F60809DBFA2228
:03000000020FC725
:100FC70078FEE4F6D8FD78007FFFE4F208DFFC75D1
:080FD700A00075819002101AC0
:100FDF00020100E493A3F8E493A34003F68001F227
:100FEF0008DFF48029E493A3F85407240CC8C33313
:100FFF00C4540F4420C8834004F456800146F6DFE2
:10100F00E4800B0102040810204080900B1EE47E48
:10101F00019360BCA3FF543F30E509541FFEE493D6
:10102F00A360010ECF54C025E060A840B8E493A39D
:10103F00FAE493A3F8E493A3C8C582C8CAC583CAC8
:10104F00F0A3C8C582C8CAC583CADFE9DEE780BE80
:010B230000D1
:00000001FF
